:020000040000FA
:0400040000EF08F011
:060008000001CED811003A
:10001800D8CF00F0E0CF01F0026E000116D80250F0
:0A00280001C0E0FF00C0D8FF100087
:100040000F0171EC1EF0000102E3D8801200D8907D
:100050001200E9CF03F0EACF04F0FACF05F0FBCFAE
:1000600006F086A538D09DA036D09EA034D09E90B4
:10007000CD90F9504444F92603D00CD014D024D0AC
:1000800081A006D0452A090E456425D0442A23D0F4
:10009000456A21D081B01FD0680E436E676B080E91
:1000A000476E442A18D0D89081B0D8804636472E63
:1000B00012D043C0E9FFEA6A46C0EFFF672B432A2C
:1000C000080E476E442A07D081B002D0440603D000
:1000D000446A456A2D8A86A35ED09DA813D09EA847
:1000E00011D09D98A8BF05D08BAF03D0A8832D80D9
:1000F00009D001EE40F0A251E926EFCFADFFA88F65
:10010000A22B98079DAA47D09EAA45D0376A096AB4
:10011000ABA203D0AB98AB8832D0ABA409D0AE5021
:10012000010E096EA8A12BD03B0EAF6EA89127D06F
:10013000AECF07F007BE9C6B01EE00F09C51E926A4
:1001400007C0EFFFA8A104D03B0EAF6EA89112D05C
:10015000A8AF10D001EE40F0A151E926EFCF08F092
:100160000750081803E0010E096E04D0A12BA19BD3
:1001700098679D88096603D02D829C2B9C9BA8AF15
:100180000AD0095208E0A89F9D98A8832D80630E8D
:10019000AF6EAD6AA88105C0FAFF06C0FBFF03C0C1
:1001A000E9FF04C0EAFF120086A509D0F2A807D033
:1001B000F2A205D0F292CF68640ECE6ECD8086A3F7
:1001C00011D0F2A80FD0F2A20DD0F292F2988B8F3C
:1001D000376A2DB007D0A8BF05D00D0EA56102D09B
:0601E000020EA52712002B
:04022E0000EF02F0EB
:0402580000EF02F0C1
:1004000000011EDE03E30D01F4D90001000100EF3D
:1004100008F01200146A1350146009D09E90B10EB7
:10042000CF6ECD809EA0FED7CD90142AF4D71200B7
:10043000898E126A115012600AD0899E0A0E136EBC
:10044000E9DF898E280E136EE5DF122AF3D7C80E76
:10045000136EE0DFEDD70DEE10F000019B51E926A1
:10046000EFCF13F00DEE10F0E926EF6A9B2B400E54
:100470009B619B6B13500D011200152C02D0176A63
:10048000000C14C018F0182A1850166201D0186A0F
:100490000D0EEA6E18501324E96EEFCF17F01750C7
:1004A000100A03E0FD0E176EFD0C186A0D0EEA6EC1
:1004B00014501324E96EEF50181A142A14501662BF
:1004C00001D0146A1704196E19521FE0150615BEE3
:1004D00002D0156602D0176A000C0D0EEA6E145099
:1004E0001324E96EEFAE03D0FE0E176EFE0C0D0E58
:1004F000EA6E14501324E96EEF50181A142A14509F
:10050000166201D0146A1906DFD7183C02D01750C2
:1005100012001768FF0C9EAA14D0ABA203D0AB98B0
:10052000AB880FD0ABA402D0AE500BD0899E0DEE9D
:1005300010F09A51E926AECFEFFF9A2B400E9A6148
:100540009A6B9B519A5D116E11AE02D0400E11262E
:1005500011522BE00DEE10F09B51E926E50EEF62F3
:1005600022D0100E136E9BC014F011C015F0400E77
:10057000166E83DF17C091FD0D01915107E0FD0A52
:1005800007E0030A05E0010A06E008D000010DD0EB
:1005900062DF00010AD012680001FF0C898E010E93
:1005A000126E0001010C57DF0001126A000CA6B2A6
:1005B000FED711C0A9FF12C0AAFFA69EA69CA680C6
:1005C000A8501200020E1D6EA69EA69CA68418C0FE
:1005D000A9FF19C0AAFF0DEE00F01BC01CF0EFCF61
:1005E000A8FF550EA76EAA0EA76EA682A6B2FED7CA
:1005F000A680A850EF6209D0020E1D6EEE50A92A07
:10060000A950D8B4AA2A1E8002D01E9002D01C2E57
:10061000E6D71EA002D0D88012001D2EE0D7D890B9
:100620001200899E020E256EA68EA69CA684A68E1A
:1006300020C0F6FF21C0F7FF22C0F8FFA688550EA4
:10064000A76EAA0EA76EA682A6980A000DEE50F01D
:1006500023C024F0EECFF5FF0F00242EFBD7550E5C
:10066000A76EAA0EA76EA682A69420C0F6FF0DEE76
:1006700050F0268023C024F00900F550EE1802E067
:10068000269002D0242EF8D726A004D09281898EFD
:10069000D8801200252ECAD7D8901200A68EA69C0C
:1006A0002250F86E2150F76EC00E2014F66E0DEE3B
:1006B00050F0400E236E0900F5CFEEFF232EFBD73E
:1006C00012003F0E18141F6E500E1F241D6E1D06C3
:1006D0001E6A1F6A1B501F5C1F501B18D8B0800A6F
:1006E00036E61D2A900E1D6219D0500E1D6E93CD58
:1006F00020F094CD21F0226A400E236E92DF0CE3AD
:10070000400E9327000E942393CD20F094CD21F03A
:10071000226AC4DF929102D0D89012000D0EEA6EC8
:100720001EC0E9FFEFCF1CF019501A1003E1030EB1
:10073000186406D00D0EEA6E1DC0E9FF1CC0EFFF65
:100740001E2A182A000E19221A221F2AC3D7D8805F
:1007500012001350176E1250166EC00E1114156E43
:10076000898E175003E1030E166407D0175005E178
:10077000010E155C0A0E16582EE317502CE1F00EF0
:10078000166029D092A10BD015C093FD16C094FD20
:1007900093CD20F094CD21F0226A80DF9291155004
:1007A00093630ED0165094630BD0176609D011C016
:1007B00018F012C019F013C01AF014C01BF081D742
:1007C00093CD20F094CD21F0226A400E236E29DFD4
:1007D000C7E2D8901200F00E136209D011C018F0D1
:1007E00012C019F013C01AF014C01BF0EBD6D88059
:1007F000120092811092899E108000018CDEFF0A07
:100800000D0103E0FE0A07E0C6D010A2C4D0040E1A
:10081000116E0EDEC0D0899E1EDE1DDE100AD8A429
:10082000BAD019DE7F0AD8A4B6D015DE7F0AD8A4C4
:10083000B2D011DE7F0AD8A4AED00DDE0A6E040E4F
:1008400000019B250C6E3F0E0C6402D0400E0C5E26
:100850000DEE10F00C50E926F00EEF140D0108E03B
:10086000100A48E0300A56E0600AD8B485D093D028
:10087000F2DD570A03E0010E116EDADDECDD160A37
:1008800003E0010E116ED4DDE6DD906F909F0AB497
:10089000908F020E00019B250C6E3F0E0C6402D05F
:1008A000400E0C5E0DEE10F00C50E926EFCF0BF071
:1008B0000D010BA00ED00BB207D09051020A09E037
:1008C000020E116EB5DD05D0020E906102D0116EE0
:1008D000AFDDC1DD906F909F0AB6908F0BA408D05A
:1008E000116A126A64DE906103D0030E116EA0DDFE
:1008F000108251D0B0DD0F6E0F9E0AB00F8EABDDAF
:100900000E6E0E9E0AB20E8EA6DD0D6E0D9E0AB400
:100910000D8E41D01DEE00F00C6A040E0C6009D063
:100920009ADDE76E0A32D8A0E69ED8B0E68E0C2A91
:10093000F4D791DD0B6E0C6A040E0C6009D08BDDD0
:10094000E76E0B32D8A0E69ED8B0E68E0C2AF4D71C
:100950000DC011F00EC012F00FC013F0080E146E8F
:10096000F8DE06E3080E0D26000E0E220F2213D02D
:10097000050E116E5DDD0FD092B10CD093CD20F03D
:1009800094CD21F0226A400E236E4BDE03E2050E69
:10099000116E4EDD109010B030D7120052BE09D04B
:1009A000D6CF0AF055500A5C565E0AC055F0D8A062
:1009B000528E1200D6CF0AF053500A5C545E0AC021
:1009C00053F0D8B012007D0E5426050E0B6E010EAA
:1009D0000C6E00EE48F052500C140DE1EF06EF3CA7
:1009E00003D0EE50EF06ED50EF50EE50EF1002E165
:1009F0000C505212ED50020EE926000EEA22D89059
:080A00000C360B2EE8D71200A2
:10100000000103D000EC02F000010D0192A320ECDE
:1010100000F0000118EC1FF074EC1FF007011CEC4D
:1010200020F05268536A546AC60ED56E2D6A0001CC
:1010300052EC20F02D862D88D08EF28EF28C306A04
:10104000316A326A336A800E426E396E3A6E3D6E94
:101050003E6E3F6E406E416E376E346E356E366E4C
:10106000386E3C6E3B6E356A366A386A3A6A3C6A5C
:101070003B6A0400D19086A503D0346AF292F288CC
:101080008DDC98DC30BE02D054D8306E31BE02D038
:101090005ED8316E32BE02D017D9326E33BE02D066
:1010A00063D9336E34BE04D001018AD9346E000195
:1010B00035BE02D050DA356E36BE02D0E4DA366E76
:1010C00037BE02D009DA376E38BE02D071DA386E18
:1010D00039BE02D021DB396E3ABE02D038DB3A6E1F
:1010E0003BBE03D095EC14F03B6E3CBE03D0E3EC6A
:1010F00011F03C6E3DBE03D01BEC17F03D6E3EBEC2
:1011000003D068EC15F03E6E3FBE03D0EDEC15F059
:101110003F6E40BE03D0B4EC19F0406E41BE03D028
:1011200090EC1BF0416E42BEABD7E7EC0FF0426E85
:10113000A7D7F9503044F92601D004D0010E486EEB
:10114000496A529052A0010C6DEC18F0000CF95055
:101150003144F92601D004D00A0E4A6E4B6A5292ED
:1011600052A2010C136A020E13603DD002EE00F091
:101170001350E926EFCF10F002EE02F0E9261050EE
:10118000EF14126E02EE08F01350E9261050EF141F
:101190000F6E12500F18116E010E0E6E0E521BE0E4
:1011A00002EE0AF01350E926EF501114106E0E50A3
:1011B00010160EE002EE08F01350E9260E50EF1A5A
:1011C0008BB506D002EE0EF01350E9260E50EF124A
:1011D000D8900E36E3D702EE0AF01350E92611C07C
:1011E000EFFF132AC0D73D6A416A3E6A3F6A0A6A26
:1011F0000B6A2B0EC26EC2B2FED7030EC4140B6E66
:10120000C3CF0AF0120E0A5C010E0B5803E279EC10
:1012100011F00001130EC26E0C6A0D6AC2B2FED745
:10122000030EC4140D6EC3CF0CF0810E0C5C010EC6
:101230000D5814E3800E0C5C020E0D580FE28BB3B8
:1012400018D0070109A303D000018B8102D000014F
:101250008B910701098300018B830BD08BA309D0ED
:101260008BA103D00701098302D007010993000174
:101270008B938BAD04D0642F02D08B9D898E86A377
:1012800022D081B008D0A8AD0DD0A32B0A0EA36345
:1012900009D0A89D07D0A36BA8BD04D0A46702D035
:1012A000010EA46FA4530FE0A42B180EA4650BD05D
:1012B000A46BF29EF292F288AB889E9A9D8A9D98CA
:1012C000AC8AF28EA88D000CF9503244F92601D078
:1012D00004D0640E4C6E4D6A529452A4010C89697C
:1012E0008A6965530EE065070F0E65150AE1653BD7
:1012F00065070F0E651504E0050E636F426A658B86
:10130000653B665307E0662F05D0050E636F426AA2
:10131000010E666F86A707D08BBD05D0050E636FE3
:10132000010E666F426AA8A51ED00B800A6A020EE3
:101330000A6017D002EE0EF00A50E926EF50D8A44A
:101340000B9002EE16F00A50E926EF50D8A40B904D
:1013500002EE18F00A50E926EF50D8A40B900A2AA2
:10136000E6D70BB0A895000CF9503344F92601D00C
:1013700005D0E80E4E6E030E4F6E529652A6010C2B
:10138000A8A71CD0A88502EE00F0A651E926EFCF51
:101390000AF002EE0EF0E9260A50EF1202EE00F01B
:1013A000A651E926EF1C0A6E02EE0EF0A651E926C0
:1013B0000A50EF12A62B020EA661A8978B95000C7F
:1013C000F9503444F92600D02DAA010C20EE67F024
:1013D00000EE73F01F0EDF14866F8629DECFEEFF5E
:1013E000E806000AFBE12D9A896B010E876F865192
:1013F000876108D0EA6A730E8725E96EEF50891B72
:10140000872BF5D7EA6A730E8725E96E8951EF625B
:101410005FD074C08BF18B495BD0000174AF37D0C3
:10142000050E0101866133D0000175AF51D03F0E2A
:101430007415040DF3CF8BF1070E7515D890E830B5
:1014400001018B13040E8B5F0001751D700BE83AD0
:101450000F0B01018C6F010E00017515E83AF00BBE
:101460000101886F8C138B510001896306D0010143
:101470008C5100018A6301D02BD08BC189F08CC1C3
:101480008AF08BC187F08CC188F0000E7FDA0001F2
:1014900074AF1ED0040E010186651AD03F0E000104
:1014A000741501018C6F75C08BF18B51606303D093
:1014B0008C51611906E00F0E8B630AD0270E8C63E6
:1014C00007D0EC0E00017615EC0AD8B442EC1DF002
:1014D0000101000C0101800CF9503744F92602D0BB
:1014E00007D035D08B8FD6CF55F0960E566E529EC4
:1014F00052AE010CF292F288A5450A6E0A44060F1C
:10150000F924D8B0FA2AF96E960E1DD08E0E1BD093
:10151000860E19D07F0E17D0780E15D0700E13D00E
:10152000690E11D0610E0FD05A0E0DD0520E0BD095
:101530004A0E09D0430E07D03C0E05D0340E03D01E
:101540002D0E01D0000ED6CF55F0566E529E52AEE3
:10155000020C8B9F800C0101F9503544F92600D014
:1015600000012DA2010C010100AF1ED040D90A6E6E
:101570000A50000119E0FF0A05E10101006B0001BA
:10158000A89F12D011EE00F004EE00F09A51E92667
:10159000E6CFEEFFE950D8B404EE00F00A2EF8D7FB
:1015A000E9CF9AF0A89F2D802D922D8C0001000C80
:1015B0003850D8A4800C9A519B1964E004EE00F0D6
:1015C0009B51E926EFAE5DD004EE00F0E926EF5026
:1015D000830A0DE0330A0FE0010A22E0030A2FE03C
:1015E0005F0A3CE0020A46E05B0A49E04AD0070194
:1015F000FAEC0FF046D08CEC0FF00AC087F00BC06D
:1016000088F087518815FF0A3CE0000EBFD912C050
:101610000AF013C00BF070EC13F0869F406A31D0D3
:101620008CEC0FF00AC087F00BC088F0875188154A
:10163000FF0A27E0010EAAD9869F406A22D08CECCF
:101640000FF00AC087F00BC088F087518815FF0A99
:1016500018E0020E9BD9869F406A13D02DEC0FF044
:101660000AC087F00BC088F087518815FF0A09E08F
:10167000868F07D00701F4EC1BF0000102D029ECA3
:101680001EF09B2B000C0101F9503644F92603D0C3
:1016900002D02ED038D000012DA4010C2D940101D0
:1016A00040390F0B0001A56F0F0E0101401500011D
:1016B000986F010EA16FA26F86A515D0040E9C6FC6
:1016C000576A985157600DD001EE41F05750E92606
:1016D000EFCF58F001EE00F0E92658C0EFFF572A8F
:1016E000F0D72D8217D08BBF02D0A8BD03D0020C3B
:1016F0000001F9D76EEC20F08BBFD6D79D882D90D6
:101700002DB003D0030C0001FBD7A8A302D0A893EF
:10171000CBD7A56B2D86000CF9503944F92600D0A3
:101720002DA6010C2D9611EE20F0E6CF0AF021EE49
:1017300040F00AC0DEFF0A060B6AE6CFDFFFDE508C
:101740000B1A0A2EFAD70B1CDF6E2D84800CF95071
:101750003A44F92601D006D09F519D6303D0A05191
:101760009E1944E02DA6010C2D9621EE40F09D51CE
:10177000E96E050E9E25EA6EEFCF0AF00AC0DEFF85
:101780009D2B000E9E239D6705D0020E9E6302D006
:101790009D6B9E6B0A060B6A9D51E96E050E9E2598
:1017A000EA6EEFCFDFFFDE500B1A9D2B000E9E235B
:1017B0009D6705D0020E9E6302D09D6B9E6B0A2E24
:1017C000EBD70B1CDF6E9D519F5D0A6E9E51A05999
:1017D0000B6E0BAE02D0020E0B260BBE05D0D00E48
:1017E0000A5C010E0B58D8A02D882D84000C00AD8A
:1017F00014D000AB0FD0020E00019C6101D0000C90
:1018000001C10BF0030E01010B6403D0100E0B6439
:101810000BD0FF0C060E0B6E07D000AB03D0040EEE
:101820000B6E02D0020E0B6E00019C510B6212D0A7
:101830000C6A0D6A01EE00F00D50E926EF500C1A0B
:101840000D2A0B500D5CF6E30C28010102E10B5050
:101850001200FF0C000C176E1438030B1A6E1D9249
:1018600016BE1D821D9416B81D841DB014D01DA275
:1018700007D017B005D00F0E1614196E1550186E3C
:101880001DA209D017A007D018C015F019C016F076
:1018900016981DB416881F0E16161DB019D01A50B2
:1018A00005E0010A06E0030A0AE011D01686169A3E
:1018B00031D0169A168616A82DD016962BD016342F
:1018C000163215321698D8B01688168A23D0120010
:1018D0001A5005E0010A09E0030A10E01AD0168642
:1018E000100E14BC161A169A15D0169A100E14BCA7
:1018F000161A168616A80ED016960CD01634163266
:1019000015321698D8B01688168A080E14BC161A06
:1019100001D01200D89015361636D89015329F5146
:10192000E96E050EA025EA6E040EEF6E58DB9F519E
:10193000E96E050EA025EA6EB00E1A10EF6E4FDBB1
:101940009F51E96E050EA025EA6E15C0EFFF47DB3B
:101950009F51E96E050EA025EA6E16C0EFFF3FDB32
:101960009D519F5D1B6E9E51A0591C6E1CAE02D0F6
:10197000020E1C261CBE06D0E10E1B5C010E1C587C
:10198000D8B02D98050E636F426A12000A6E0F0ED2
:1019900000018815136E8751126E0F6A020E0F60D8
:1019A0009CD10E68010E106E1052D8B494D10E2A3C
:1019B00002EE00F00F50E926EF1C1014D8B488D1C5
:1019C0000F50400DF3CFD9FFF4CFDAFF100ED92618
:1019D000070EDA22080E0E02F350D926000EDA2284
:1019E0000EA015D0080ED95E000EDA5ADCCF0BF02F
:1019F000DD501C940BBC1C841C960BBE1C861CA6C4
:101A000002D01CA404D0080ED926000EDA22DECFA4
:101A100014F0070EDF14156ED9CF1AF0DACF1BF0D1
:101A2000030ED926000EDA22DECF16F0DFCF1DF02E
:101A30000F0EDE14176EDECF18F0DFCF1EF00F0E84
:101A4000DE14196E1AC0D9FF1BC0DAFFDECF0BF00F
:101A50001C940BBC1C841C960BBE1C86DFCF0CF0A8
:101A6000DCCF1FF0DD501F38070B1F6E0B38030B48
:101A70000A6244D01250146241D0135015623ED015
:101A8000030E0C143BE01C9288B91C82020EDFBED0
:101A90001C1A0A620ED00AC020F0299029921CB2AA
:101AA00029820EC021F00FC022F01050AAEC13F0D2
:101AB00025D01CB414D01CA612D00EA010D00AC081
:101AC00020F029901CB4298029821CB229920EC0D2
:101AD00021F00FC022F01050AAEC13F00FD00AC072
:101AE00020F029901CB4298029921CB229820EC0B2
:101AF00021F00FC022F01050AAEC13F0030ED926EB
:101B0000000EDA22DFCF0DF0D8900C32D8900C32D4
:101B1000030E0C1468E01C9288B91C82030E0C148E
:101B2000010A05E0030A06E0010A06E05CD01CB2E7
:101B300003D059D01CB257D00DAE2FD01250166220
:101B400052D0135017624FD0020E0DBC1C1A1CB499
:101B500014D01CA612D00EA010D00AC020F02990DC
:101B60001CB4298029821CB229920EC021F00FC01A
:101B700022F01050AAEC13F036D00AC020F02990C1
:101B80001CB4298029921CB229820EC021F00FC0FA
:101B900022F01050AAEC13F026D01250146203D099
:101BA0001350151808E0125018621DD01350196216
:101BB0001AD01EAE18D001EE82F00F50E926EFCFFA
:101BC00011F01CA203D01050111202D0101C1116DB
:101BD00001EE82F00F50E92611C0EFFF02EE16F081
:101BE000E9261050EF12020ED926000EDA22DFCFBE
:101BF0000DF0D8900C32D8900C32030E0C1468E023
:101C00001C9288B91C82030E0C14010A05E0030A19
:101C100006E0010A06E05CD01CB203D059D01CB229
:101C200057D00DAE2FD01250186252D013501962F7
:101C30004FD0020E0DBC1C1A1CB414D01CA612D01E
:101C40000EA010D00AC020F029901CB4298029824F
:101C50001CB229920EC021F00FC022F01050AAEC45
:101C600013F036D00AC020F029901CB429802992A4
:101C70001CB229820EC021F00FC022F01050AAEC35
:101C800013F026D01250146203D01350151808E038
:101C9000125016621DD0135017621AD01DAE18D004
:101CA00001EE84F00F50E926EFCF11F01CA203D013
:101CB0001050111202D0101C111601EE84F00F50BA
:101CC000E92611C0EFFF02EE18F0E9261050EF12DE
:101CD000D890103669D60F2A61D6125012009F5143
:101CE000E96E050EA025EA6E0B0EEF6E78D99F51B6
:101CF000E96E050EA025EA6EED0EEF6E70D99F51CC
:101D0000E96E050EA025EA6E0B0EEF6E68D99F51A5
:101D1000E96E050EA025EA6E7F0EEF6E60D99F5129
:101D2000E96E050EA025EA6E310EEF6E58D9143813
:101D3000E8441F0B156E143A1442F80E1416030EE5
:101D400013141412D8901436700E141A1480149EA2
:101D5000D8901332D89013329F51E96E050EA0250A
:101D6000EA6E010EEF6E3BD99F51E96E050EA0257C
:101D7000EA6E13C0EFFF33D99F51E96E050EA0251F
:101D8000EA6E14C0EFFF2BD99F51E96E050EA02516
:101D9000EA6E15C0EFFF23D99F51E96E050EA0250D
:101DA000EA6EEF6A1CD99F51E96E050EA025EA6E16
:101DB000EF6A15D99D519F5D156E9E51A059166E03
:101DC00016AE02D0020E162616BE06D0E10E155C27
:101DD000010E1658D8B02D98050E636F426A120096
:101DE000136E146886AF1AD01038E8461F0B1F0B0D
:101DF000176E1238E8461F0B1F0B186E070E1016D1
:101E000012160F50116227D01050126224D0146A9B
:101E10001750186220D0010E146E1DD01038030B1D
:101E2000176E1238E840E8423F0B030B186E17504C
:101E3000186211D00F0E10161214166E1150156E76
:101E40000F50156208D01050166205D0146A12B8EF
:101E5000142A1350141A145012009B2B04EE00F095
:101E60009B51E926EF500B0A03E00A680B68FF0C50
:101E70009B2B04EE00F09B51E926EF507F0A03E014
:101E80000A680B68FF0C9B2B04EE00F09B51E926BF
:101E9000EF38070B030A03E00A680B68FF0C9B2B63
:101EA00004EE00F09B51E926070EEF14010A03E04F
:101EB0000A680B68FF0C9B2B04EE00F09B51E9268F
:101EC000EFCF0AF00AAC03D00A680B68FF0CD89079
:101ED0000A36D8900A369B2B04EE00F09B51E92677
:101EE000EFCF0BF0700E0B1AD8900B32030E0B14C1
:101EF0000A120B3A0B461F0E0B169B2B04EE00F03A
:101F00009B51E926EFCF0CF00C3A0C42F80E0C1660
:101F10000C500B120A50120004EE00F09B51E926FF
:101F2000EFCF0CF09B2B04EE00F09B51E926D890EC
:101F3000EF340A6E9B2B04EE00F09B51E926EFCFA5
:101F40000DF004EE00F0E9263F0EEF140B6E0E903C
:101F50000DBC0E80030E0C14020A05E0030A0DE00E
:101F6000010A1EE032D00EB003D00A680B68FF0CE5
:101F70000A900DBA0A800B8E28D00EB00BD00DBA85
:101F800002D00DA804D00DAA05D00DA803D00A6870
:101F90000B68FF0CD8900B320A320B960B8C15D0C5
:101FA0000EA003D00A680B68FF0CD8900B320A32DF
:101FB0000BB60AD00AC00FF00BC010F0070121D8F1
:101FC0000A680B680001FF0C0B960A501200425081
:101FD000D8A4800C63C064F08B8D899E800C9F2BED
:101FE000000EA0239F6705D0020EA06302D09F6B56
:101FF000A06B120009A503D00001A66BA887000101
:102000001200070E1014166E0F50156EF80E155CA8
:10201000030E1658D8A0D2D0FC0E155C030E16582D
:10202000D8B0CCD0030E0F14146E10B81484116AFB
:10203000020E1160BED01268010E136E1352D8B496
:10204000B6D0122A1150400DF3CFD9FFF4CFDAFFEA
:10205000100ED926070EDA22080E1202F350D926E6
:10206000000EDA22DECF17F0DF38030B196E0F0EE9
:10207000DE14186E18BC98D0030E1C6ED89018325F
:1020800017321C2EFBD7186A070E1716DECF1AF070
:102090001B901ABC1B80030E1A141BE0175014620D
:1020A00018D009A70AD01BA008D0195206E002EEEA
:1020B0000EF01150E9261350EF1209A90AD01BB0F7
:1020C00008D0196606D002EE0EF01150E926135022
:1020D000EF12DE50DECF17F0DF380F0B196E1B90BA
:1020E00019B61B80030E19160F0EDE14186E030EA0
:1020F0001C6ED890183217321C2EFBD7186A070EA8
:1021000017160C0E1A141BE01750146218D009A7EA
:102110000AD01BB008D0195206E002EE16F011509A
:10212000E9261350EF1209A90AD01BA008D019669E
:1021300006D002EE16F01150E9261350EF12DECF52
:1021400017F0DF380F0B196E1B9019B61B80030EAA
:1021500019160F0EDF14186E030E1C6ED89018326D
:1021600017321C2EFBD7186A070E1716300E1A14DA
:102170001BE01750146218D009A70AD01BB008D072
:10218000195206E002EE18F01150E9261350EF1232
:1021900009A90AD01BA008D0196606D002EE18F0D3
:1021A0001150E9261350EF12D890133647D7112A51
:1021B0003FD7180E091502E00001A885070112009B
:1021C0001C6E020EEA6E1BC0E9FF1C461C461C4436
:1021D000060FF924D8B0FA2AF96EEF6A000E000053
:1021E0003BD00A0EEF6E000E37D0140EEF6E000ECD
:1021F00033D0230EEF6E000E2FD0320EEF6E000E96
:102200002BD0410EEF6E000E27D0500EEF6E000E59
:1022100023D0640EEF6E000E1FD07D0EEF6E000E09
:102220001BD0960EEF6E000E17D0C80EEF6E000E8C
:1022300013D02C0EEF6E010E0FD0900EEF6E010E2C
:102240000BD0F40EEF6E010E07D0580EEF6E020E9B
:1022500003D0200EEF6E030EEC6E12001C6E020E09
:10226000EA6E1BC0E9FF1C461C46F9501C44F926C7
:10227000E80EEF6E030E3BD0DC0EEF6E050E37D08E
:10228000D00EEF6E070E33D0B80EEF6E0B0E2FD0C0
:10229000A00EEF6E0F0E2BD0880EEF6E130E27D010
:1022A000700EEF6E170E23D0280EEF6E230E1FD088
:1022B000E00EEF6E2E0E1BD0500EEF6E460E17D0B6
:1022C000C00EEF6E5D0E13D0300EEF6E750E0FD098
:1022D000A00EEF6E8C0E0BD0100EEF6EA40E07D07A
:1022E000800EEF6EBB0E03D0600EEF6EEA0EEC6E4A
:1022F000120086B93DD0070109A13AD0F29E900E96
:102300000E6E010E0F6E106A020E0001106010D0EA
:102310000EC013F00FC014F002EE08F01050E926C2
:10232000EF5041EC1EF00E2A000E0F22102AECD7BF
:10233000602B000E612362230EC013F00FC014F057
:10234000605141EC1EF00E2A000E0F220EC013F059
:102350000FC014F0615141EC1EF00E2A000E0F2246
:102360000EC013F00FC014F0625141EC1EF08689CC
:10237000116A126A2B0EC26E0001C2B2FED7030EA2
:10238000C414126EC3CF11F01D0E115C010E125851
:1023900009E2899E640E136E08D8898E640E136E4E
:1023A00004D8E6D7D190FF001200146A13501460CD
:1023B00009D0A192B10EB36EB180A1A2FED7B190A7
:1023C000142AF4D71200F9503C44F92602D006D062
:1023D0002FD05B6A020E5B604CD1010C02EE0EF056
:1023E0005B50E926EF50D8B442D102EE00F05B50CA
:1023F000E926EF50D8B43BD15968010E5A6E5A52B3
:10240000D8B435D1592A02EE0EF05B50E926EFCF51
:102410005CF002EE00F0E926EF505C165A505C14B6
:10242000D8B422D102EE0EF05B50E9265A1CEF160A
:102430002DA8020C5B50400DF3CFD9FFF4CFDAFF8B
:10244000100ED926070EDA22080E5902F350D926AB
:10245000000EDA22DECF5DF05E6ADFCF5EF0DECF07
:102460000AF0DFCF0BF0DECF0CF0DECF0DF002EE86
:1024700008F05B50E9265A50EF145E88D8B45E9895
:102480000A38030B03E1A8A564D0EED00D38070B82
:1024900060E1A8B55ED002EE04F05B50E9265A5028
:1024A000EF1416E002EE04F05B50E9265A1CEF161A
:1024B00002EE10F05B50E9265A50EF14D880D8B4E1
:1024C000D89003E25EB8D0D044D05EB842D0CCD031
:1024D00002EE14F05B50E9265A50EF1424E102EEAC
:1024E00010F05B50E9265A1CEF165EA813D002EEDE
:1024F00010F05B50E9265A50EF12030E0C14030A39
:1025000028E00DC00EF059C00FF05BC010F05A501B
:10251000B1D8AAD00DC00EF059C00FF05BC010F0BA
:102520005A50A8D8A1D002EE10F05B50E9265A50BC
:10253000EF14D880D8B4D89003E25EB803D009D0A5
:102540005EB807D002EE14F05B50E9265A1CEF1675
:102550008BD0030E0C14010A07E0030A08E0010AFD
:1025600008E0030A4BE005D05EB803D047D05EB860
:1025700045D05DC096F05EC097F0000E5EB8010ECB
:102580000BAE04D0000A5E98D8B45E880A38030BFC
:1025900027E102EE0CF05B50E926EFCF0EF05EACC7
:1025A00003D05A500E1A08D05EB802D05A1C0E162C
:1025B0005EA802D05A500E125EAE07D059A003D0CA
:1025C0005A500E1202D05A1C0E165A500E145E8823
:1025D000D8B45E9802EE0CF05B50E9260EC0EFFF17
:1025E0000AC014F01D905DC015F05EC016F0595081
:1025F0002BEC0CF096C05DF097C05EF0A8B534D01F
:10260000D8900C32D8900C32030E0C14010A07E05B
:10261000030A08E0010A08E0030A0CE005D05EB8EE
:1026200003D008D05EB806D002EE16F05B50E92663
:102630005A50EF12D8900C32D8900C32030E0C1472
:10264000010A07E0030A08E0010A08E0030A0CE0B7
:1026500005D05EB803D008D05EB806D002EE18F000
:102660005B50E9265A50EF12D8905A36C8D65B2AEA
:10267000B1D6000C116E0F0E0E14126E0E38070B31
:10268000136E020A02E013662AD0080E1002F350FD
:102690000F24146E125207E0D89014341A0F1B6ED8
:1026A00012508EDD16D0020E136209D002EE1AF01F
:1026B000D8901434E9260A0EEE6EEF6A0AD013663B
:1026C00008D002EE1AF0D8901434E926010EEE6E0E
:1026D000EF6A02EE14F01050E9261150EF121200CA
:1026E0000A500B14FF0AD8B4120027EE10F0116A3A
:1026F000020E11602ED00F6A010E106E105227E0EC
:10270000DECF0CF0DFCF0DF00DBE19D0070E0D1689
:10271000DECF0EF0129088B912800E38030B0FE155
:102720000A500C620CD00B500D6209D02C9012B0E4
:102730002C800C0E11242A6E10505BEC18F0060E43
:10274000D926000EDA220F2AD8901036D7D7112AB0
:10275000CFD71200236E29B013D02C9029B22C8031
:10276000080E22242A6E23505BEC18F002EE0EF0C5
:102770002250E9262350EF12050E636F426AD4D02F
:102780002066D2D021B007D002EE14F02250E92604
:10279000231CEF1608D002EE14F02250E926D89040
:1027A0002330FF0AEF1621B027D02C8029B22C90BD
:1027B000080E22242A6E23505BEC18F02C8029B2DC
:1027C0002C90060E22242A6E23505BEC18F02C90DD
:1027D00029B22C80080E22242A6ED89023345BEC78
:1027E00018F02C9029B22C80060E22242A6ED89044
:1027F00023345BEC18F098D029B21FD02C90080E2F
:1028000022242A6E23505BEC18F02C90060E222412
:102810002A6E23505BEC18F02C90080E22242A6EAE
:10282000D89023305BEC18F02C90060E22242A6EF0
:10283000D89023305BEC18F077D0D9CF27F0DACFDF
:1028400028F02250400DF3CFD9FFF4CFDAFF130E5A
:10285000D926070EDA22080E2102F350D926000EDF
:10286000DA220F0EDF14256E255006E0050A04E07B
:102870000F0A02E0050A27E12C9025B22C80080EF1
:1028800022242A6E23505BEC18F02C9025B22C8069
:10289000060E22242A6E23505BEC18F02C9025B0F3
:1028A0002C80080E22242A6ED89023305BEC18F07E
:1028B0002C9025B02C80060E22242A6ED89023302E
:1028C0005BEC18F02DD02C80080E22242A6E2350A9
:1028D0005BEC18F02C80080E22242A6ED89023304E
:1028E0005BEC18F0080ED95E000EDA5A5F0EDF14AA
:1028F00017E0060E2114266E080E2202F35026243D
:10290000246E02EE1AF0D8902434E926010EEE6E01
:10291000EF6A02EE14F02250E926D8902330EF122D
:1029200027C0D9FF28C0DAFF1200F9503B44F9262E
:1029300002D01AD030D0AA6B020EAA61C8D002EE23
:102940000EF0AA51E926EFCFACF002EE00F0E92636
:10295000EF1CAC15D8B4B9D05F68010EAB6FAB53A8
:10296000D8B4B3D05F2A010C02EE0EF0AA51E926CA
:10297000EFCFACF002EE00F0E926EF1CAC17AB5144
:10298000AC15D8B49FD002EE0EF0AA51E926AB1DCB
:10299000EF16A8A53DD02DA8020CAA51400DF3CFEB
:1029A000D9FFF4CFDAFF110ED926070EDA22080E6E
:1029B0005F02F350D926000EDA22DDCF0BF00BBCFC
:1029C00081D00B38030B7EE1DECF0CF00D6ADECF39
:1029D0000DF0DFCF0EF00F900EBE0F8002EE08F06C
:1029E000AA51E926AB51EF140D88D8B40D980FA069
:1029F00004D0000A0D98D8B40D88100E146E1D90E6
:102A00000CC015F00DC016F05F502BEC0CF05AD036
:102A1000AA51400DF3CFD9FFF4CFDAFF110ED9261A
:102A2000070EDA22080E5F02F350D926000EDA22D2
:102A3000DECFADF0DECFAEF0DECFAFF00F0EAF15D4
:102A4000B06FAF39070BAF6F030EAE150CE0AFC020
:102A500010F0B0C011F0ADC012F05FC013F0AAC00A
:102A600014F0AB513FD9DCCF0AF0D890AE33D890F8
:102A7000AE33030EAE150EE00AAE0CD0AFC010F0B0
:102A8000B0C011F0ADC012F05FC013F0AAC014F0D6
:102A9000AB5128D9DE50DCCF0AF0D890AE33D890B5
:102AA000AE33030EAE150EE00AAE0CD0AFC010F080
:102AB000B0C011F0ADC012F05FC013F0AAC014F0A6
:102AC000AB5110D9D890AB374AD7AA2B35D7000CC9
:102AD000F9503E44F92602D012D01FD0B36B020E3B
:102AE000B3617AD002EE16F0B351E926EF5072E0EE
:102AF000B169010EB26FB2536DE0B12B010C02EE61
:102B00000EF0B351E926B251EF1461E102EE16F076
:102B1000B351E926B251EF145AE02DA8020C02EE8F
:102B200016F0B351E926B21DEF16B351400DF3CFA5
:102B3000D9FFF4CFDAFF100ED926070EDA22080EDD
:102B4000B103F350D926000EDA22DCCF0AF0030ECF
:102B5000D926000EDA22DECF0BF00C6A3F0EDF140E
:102B60000C6EDFCF0DF001EE82F0B351E926B251C9
:102B7000EF140C88D8B40C980E900ABE0E8002EEAA
:102B800000F0B351E926B251EF140EE00EB00CD0B4
:102B90000A38030B09E102EE0CF0B351E926B251F9
:102BA000EF140C88D8B40C98A8A507D00D38030BE7
:102BB0000F6E0F6602D0100E0D6E0DC014F01D804A
:102BC0000BC015F00CC016F0B1512BEC0CF0D890E6
:102BD000B23791D7B32B83D7800CF9503F44F926F5
:102BE00002D012D01FD0B56B020EB5617AD002EEC2
:102BF00018F0B551E926EF5072E0B669010EB46FD6
:102C0000B4536DE0B62B010C02EE0EF0B551E9267F
:102C1000B451EF1461E102EE18F0B551E926B45158
:102C2000EF145AE02DA8020C02EE18F0B551E92677
:102C3000B41DEF16B551400DF3CFD9FFF4CFDAFF35
:102C4000100ED926070EDA22080EB603F350D92645
:102C5000000EDA22DCCF0AF0050ED926000EDA22A9
:102C6000DECF0BF00C6A3F0EDF140C6EDFCF0DF0E1
:102C700001EE84F0B551E926B451EF140C88D8B4B4
:102C80000C980E900ABE0E8002EE00F0B551E926B7
:102C9000B451EF140EE00EB00CD00A38030B09E16A
:102CA00002EE0CF0B551E926B451EF140C88D8B4FB
:102CB0000C98A8A507D00D38030B0F6E0F6602D035
:102CC000100E0D6E0DC014F01D800BC015F00CC061
:102CD00016F0B6512BEC0CF0D890B43791D7B52B39
:102CE00083D7800C156E02EE08F01450E9261550BB
:102CF000EF147EE0080E1402F3501324166E1052E7
:102D000003E0020E106208D0D89016341A0F1B6E22
:102D10001150E0EC10F00CD0104C03D0030E1062F8
:102D200007D0D89016341A0F1B6E11502EEC11F0EC
:102D300002EE1AF0D8901634E926EECF19F0EECF55
:102D40001AF01050020A07E0010A10E0030A2DE011
:102D5000010A36E06BD019501A1008E102EE06F0B5
:102D60001450E9261550EF12D890120002EE14F01C
:102D70001450E9261550EF1459E102EE06F01450F4
:102D8000E9261550EF1A02EE1AF0D8901634E9260B
:102D900019C0EEFF1AC0EEFF02EE14F01450E9263F
:102DA0001550EF12010E186E41D019501A1008E19B
:102DB00002EE06F01450E9261550EF12D8901200DA
:102DC00002EE06F01450E9261550EF1202EE1AF04A
:102DD000D8901634E92619C0EEFF1AC0EEFF02EEB5
:102DE00014F01450E9261550EF12010E186E1ED083
:102DF0001050020A07E0010A05E0030A09E0010A8F
:102E000007E013D002EE14F01450E926151CEF165B
:102E100002EE14F01450E9261550EF1406E102EE0C
:102E200006F01450E926151CEF16186A1850D880C1
:102E3000D8B4D8901200F9503D44F92601D005D0FD
:102E4000B76B020EB761ADD0010C02EE14F0B751B2
:102E5000E926EF50D8B4A3D00B68010E0A6E0A52CF
:102E6000D8B49DD00B2A02EE14F0B751E9260A50CF
:102E7000EF14D8B491D0B751400DF3CFD9FFF4CFB0
:102E8000DAFF100ED926070EDA22080E0B02F350D5
:102E9000D926000EDA22DCCF0CF0DCCF0EF0DCCF2E
:102EA0000DF00D38070B0F6E02EE1AF0080EB70387
:102EB000F3500B24D890E834E926EE06000EEF5AC2
:102EC00002EE1AF0080EB703F3500B24D890E83442
:102ED000E926EE50EF1060E102EE00F0B751E9266E
:102EE000EF1C0A1447E00CAC19D0080ED926000ECE
:102EF000DA220D38F00B0D6E0F0EDF140D26080EC2
:102F0000D95E000EDA5A0FC010F00DC011F00BC0E0
:102F100012F0B7C013F00A5045D83ED00F50020A45
:102F200003E0030E0F6213D002EE14F0B751E9264E
:102F30000A1CEF160FC010F00F0E0D14116E126A5E
:102F40000BC013F0B7C014F00A50CCDE10D00F52F3
:102F500002E00F2C0CD002EE14F0B751E9260A1C47
:102F6000EF1602EE06F0B751E9260A1CEF16A8A5E7
:102F700013D012D002EE14F0B751E9260A1CEF1656
:102F800002EE04F0B751E9260A50EF1202EE0EF0FD
:102F9000B751E9260A50EF12D8900A3660D7B72BFE
:102FA00050D7800C146E02EE06F01350E926196A11
:102FB000EFCF18F0125005E01A6ED89018321A2E82
:102FC000FCD7196A030E18161114186212D02C902F
:102FD00011B42C80060E13242A6E14506CD82C9039
:102FE00011B62C80060E13242A6ED890143463D8A0
:102FF00011D02C9011B02C80060E13242A6E145080
:103000005AD82C9011B22C80060E13242A6ED89018
:10301000143451D811380F0B116E080E1302F350EF
:103020001224156E02EE14F01350E926141CEF164C
:103030001050020A03E0010A1BE033D0D890153487
:103040001A0F1B6E1150E0EC10F002EE1AF0D8903F
:103050001534E926EECF16F0EECF17F01650171004
:1030600020E002EE14F01350E9261450EF1219D0AC
:10307000D89015341A0F1B6E11502EEC11F002EE81
:103080001AF0D8901534E926EECF16F0EECF17F0EF
:103090001650171006E002EE14F01350E9261450F3
:1030A000EF1202EE1AF0D8901534E92616C0EEFFA2
:1030B00017C0EEFF12002B6E020EEA6E2AC0E9FF67
:1030C000D8902B50EF14D8A4D8802CA003D02B502C
:1030D000EF1202D02B1CEF1612000A6A020E0A60D1
:1030E00042D102EE06F00A50E926EFCF0BF002EED5
:1030F00000F0E926EF1C0B1602EE12F00A50E9264A
:10310000EF500B1A0A6691D002EE00F00A50E92641
:10311000EFB005D00BA08A960BB08A8607D002EEDE
:1031200002F00A50E926EF9081B6EF8002EE00F03F
:103130000A50E926EFB205D00BA289960BB2898618
:1031400007D002EE02F00A50E926EF9280B6EF8235
:1031500002EE00F00A50E926EFB405D00BA48A94E1
:103160000BB48A8407D002EE02F00A50E926EF94ED
:1031700081B4EF8402EE00F00A50E926EFB605D0E4
:103180000BA689940BB6898407D002EE02F00A5090
:10319000E926EF9680B4EF8602EE00F00A50E926A9
:1031A000EFB805D00BA88B920BB88B8207D002EE3C
:1031B00002F00A50E926EF9882B2EF8802EE00F0A2
:1031C0000A50E926EFBA05D00BAA89920BBA898278
:1031D00007D002EE02F00A50E926EF9A80B2EF8A99
:1031E00002EE00F00A50E926EFBC05D00BAC8B9044
:1031F0000BBC8B8007D002EE02F00A50E926EF9C50
:1032000082B0EF8C02EE00F00A50E926EFBE05D046
:103210000BAE89900BBE898098D002EE02F00A5066
:10322000E926EF9E80B0EF8E90D002EE00F00A50BB
:10323000E926EFB005D00BA08B9A0BB08B8A07D094
:1032400002EE02F00A50E926EF9082BAEF8002EE19
:1032500000F00A50E926EFB205D00BA28A9E0BB20D
:103260008A8E07D002EE02F00A50E926EF9281BE64
:10327000EF8202EE00F00A50E926EFB405D00BA46D
:103280008B980BB48B8807D002EE02F00A50E92627
:10329000EF9482B8EF8402EE00F00A50E926EFB610
:1032A00005D00BA68A9C0BB68A8C07D002EE02F0E2
:1032B0000A50E926EF9681BCEF8602EE00F00A5034
:1032C000E926EFB805D00BA88B960BB88B8607D0F4
:1032D00002EE02F00A50E926EF9882B6EF8802EE7D
:1032E00000F00A50E926EFBA05D00BAA8A9A0BBA69
:1032F0008A8A07D002EE02F00A50E926EF9A81BAD4
:10330000EF8A02EE00F00A50E926EFBC05D00BACC4
:103310008B940BBC8B8407D002EE02F00A50E92696
:10332000EF9C82B4EF8C02EE00F00A50E926EFBE6B
:1033300005D00BAE8A980BBE8A8807D002EE02F049
:103340000A50E926EF9E81B8EF8E02EE00F00A5097
:10335000E926EF500B1602EE02F00A50E9260B5058
:10336000EF1A0A2ABBD61200F9504044F92602D0BF
:10337000DBD04DD1800E386E2C9AB86B200EB86120
:1033800048D1080EB803F350900FB96F070EBA6B0F
:10339000BA23B9C0D9FFBAC0DAFFDFAE38D1040E04
:1033A000D924E16E000EDA20E26E2C98E6CF0BF005
:1033B000E7CF0CF00D6AE7BC0D2A0E90E7B80E803F
:1033C000DFB802D0E7AE39D0DFA802D086BF04D084
:1033D000DFB838D086BF36D00C980BC00FF00CC0C9
:1033E00010F087C011F088C012F00D50F0EC0EF014
:1033F00014C00AF00ABE26D001EE62F0B851E926E8
:10340000EF9C0AB00CD001EE62F0E926EF9A0AB008
:10341000EF8A01EE62F0E926EF900AB0EF8001EE4C
:1034200062F0B851E926EF900AB0EF800EA00AD002
:1034300001EE62F0E926EF8C05D001EE62F0B851A2
:10344000E926EF80060ED924E16E000EDA20E26E46
:10345000E6CF0BF0E7CF0CF00D6AE7BC0D2A0E901B
:10346000E7B80E80DFB602D0E7AE30D0DFA602D0DC
:1034700086BF04D0DFB62FD086BF2DD00C980BC0EE
:103480000FF00CC010F087C011F088C012F00D5082
:10349000F0EC0EF014C00AF00ABE1DD001EE62F08E
:1034A000B851E926EFA004D001EE62F0E926EF8AD8
:1034B00001EE62F0B851E926EF920AB0EF820EA059
:1034C0000AD001EE62F0E926EF8C05D001EE62F041
:1034D000B851E926EF820E92DFBC0E822CBA06D0DC
:1034E000B85199D82C98D8B02C8809D001EE62F048
:1034F000B851E926EF9801EE62F0E926EF9601EE69
:1035000062F0B851E926EFB62C8A0EB22C9A2CA89C
:103510007DD0D9CFE1FFDACFE2FFE4BE05D001EEE6
:1035200062F0E926EFB872D02DA8010CB9C0D9FF1E
:10353000BAC0DAFFD9CFE1FFDACFE2FF070EE41419
:103540000FE0010A11E0030A13E0010A15E0070A7F
:1035500017E0010A19E0030A1CE0010A1FE022D06B
:10356000010E0A6E0B6A1ED0050E0A6E0B6A1AD087
:103570000A0E0A6E0B6A16D0320E0A6E0B6A12D051
:10358000640E0A6E0B6A0ED0F40E0A6E010E0B6EFC
:1035900009D0E80E0A6E030E0B6E04D0880E0A6E78
:1035A000130E0B6EE738E8461F0B0F0B0C6E0A501C
:1035B0000C02F3CF0DF0F4CF0EF00F6A0B500C029B
:1035C000F3500E26F4500F220CAE04D00A500E5EBB
:1035D0000B500F5A0BAE02D00C500F5E0D500E1058
:1035E0000F1012E003EE00F0030EB803F350E926CB
:1035F0000DC0EEFF0EC0EEFF0FC0EEFF01EE62F059
:10360000B851E926EF8802D0B851BBD8020CB82BCC
:10361000B5D6386A800C0F6E1190080E0F02F35069
:10362000900FE16E070EE26AE22201EE62F00F50A7
:10363000E926D890E73006E3EFB002D0EFA206D03B
:10364000118004D0EFA002D0EFB21180D890E73003
:10365000030B106E105007E0010A1DE0030A33E06F
:10366000010A41E05BD011A013D0EFBC07D011B02C
:1036700003D0EFB403D007D0EFB405D0EF86EF84CA
:10368000EF9CD8801200EFB649D0EF86D8801200A8
:10369000EF96EF9443D011B013D0EFBC07D011B028
:1036A00003D0EFB403D007D0EFB405D0EF86EF948A
:1036B000EF9CD8801200EFB631D0EF86D880120090
:1036C000EF96EF842BD0EFBC07D011B003D0EFB44E
:1036D00003D024D0EFB422D011A0EF9411B0EF8426
:1036E000EF9CD880120011A017D0EFBA02D0D8906A
:1036F0001200EFBC07D011B003D0EFB403D007D055
:10370000EFB405D0EF86EF84EF9CD8801200EFB6BF
:1037100005D0EF86D8801200EF96EF94D890120073
:10372000F9504144F92602D006D024D0BB6B200EBC
:10373000BB6126D0010C01EE62F0BB51E926EFA877
:103740001DD003EE00F0030EBB03F350E926EE0696
:10375000000EEE5AEF5A03EE00F0030EBB03F350D7
:10376000E926EE50EE10EF1009E101EE62F0BB51D8
:10377000E926EF982DA8020CBB5103D8BB2BD7D755
:10378000800C106E080E1002F350900FE16E070EC1
:10379000E26AE222E7AA10D0020EE126000EE2223F
:1037A000E6CF11F0126AE7CF12F011C013F012C089
:1037B00014F06FEC0EF017D0020EE126000EE2229C
:1037C000E6CF11F0126A0F0EE714126E1288E7CFDF
:1037D00013F013C014F01D8011C015F012C016F0C4
:1037E000000E2BEF0CF0120009A3120000019B2B1E
:1037F0009B2B04EE00F09B51E9267C0EEF625AD021
:103800009B2B04EE00F09B51E926EFCF0CF09B2B95
:103810009B2B04EE00F09B51E926EFCF0BF09B2B86
:1038200004EE00F09B51E926D890EF340A6E0B3479
:103830000B320A320A500101606304D00B506163FD
:1038400001D00BD000018BA307D00F0E0A6204D069
:10385000270E0B6201D001D0120000019B2B9B2B85
:10386000FC0E0C14200A0BE0080A09E0040A11E01F
:103870004C0A19E0080A17E00C0A19E01BD00CC02A
:103880000DF00AC00EF00BC00FF015D8010EA9D92B
:1038900011D00CC00DF00AC00EF00BC00FF00BD809
:1038A000010E9FD907D0EED8400E9BD903D0EAD89D
:1038B000400E97D9120011EE20F00E0EE66EE70EC4
:1038C000E66E0E0EE66E7C0EE66E0DC0E6FFE66A54
:1038D000D8900E360F36D8900E320FC0E6FF0EC0CD
:1038E000E6FFE66A166A04EE00F09B51E926EFCF88
:1038F00014F014C013F013380F0B136E9B2B04EE4F
:1039000000F09B51E926EFCF15F015C012F0129E82
:1039100014B0128E1790125013100AE1040E126E9A
:10392000136AE96E070E1324EA6EEFCF16F01780C4
:10393000135003E1050E126412D0135010E1090E6A
:1039400012600DD0060E125E000E135A1250E96E70
:10395000070E1324EA6EEFCF16F0178080D0100EFA
:10396000126202D0135205E0110E12620FD01366DC
:103970000DD00C0E125E000E135A1250E96E070E97
:103980001324EA6EEFCF16F0178069D01B0E126277
:1039900002D0135205E01C0E12620FD013660DD038
:1039A000150E125E000E135A1250E96E070E132404
:1039B000EA6EEFCF16F0178052D06F0E126214D05D
:1039C000136612D0660E125E000E135A1250E96E84
:1039D000070E1324EA6EEFCF16F08BA303D01692D6
:1039E0008BB1168217803BD0135003E16F0E126427
:1039F00013D0135011E1730E12600ED06E0E125ED2
:103A0000000E135A900E1224E96E080E1320EA6E6F
:103A1000EFCF16F0178023D0135002E112AE10D072
:103A200013660ED0800E125E000E135A100E122472
:103A3000E96E070E1320EA6EEFCF16F017800FD055
:103A400013520DE0020E13600AD01306900E1224DA
:103A5000E96E070E1320EA6EEFCF16F0178014926E
:103A600016BE148214C0E6FF15C0E6FF7F0E1614C2
:103A7000E66EE66AE66A17A003D0050E636F426A37
:103A8000A9811200119086A50CD00C0E76150C0A97
:103A9000D8A41200030E7615106E77C00FF078C010
:103AA0000DF086A31DD004EE00F09B51E926EFCF68
:103AB00010F09B2B04EE00F09B51E926EFCF0FF0A6
:103AC0000F9E10B00F8E9B2B04EE00F09B51E92649
:103AD000EFCF0DF00D9E10B20D8E10380F0B106E43
:103AE00010502FE1200E0F602CD0100E0F6202D06C
:103AF000105205E0110E0F620ED010660CD00C0EA5
:103B00000F5E000E105A0F50E96E070E1024EA6E79
:103B10000DC0EFFF58D01B0E0F6202D0105205E00F
:103B20001C0E0F6250D010664ED0150E0F5E000EA8
:103B3000105A0F50E96E070E1024EA6E0DC0EFFF09
:103B400042D06F0E0F6213D0106611D0660E0F5E5A
:103B5000000E105A0F50E96E070E1024EA6E800E08
:103B60000D10EF6E8B910DB28B8111802CD0105007
:103B700002E10FAE14D0106612D0800E0F5E000E60
:103B8000105A100E0F24E96E070E1020EA6E0DC0B9
:103B9000EFFF100E0F26000E1022118014D01052CD
:103BA00011E0020E10600ED01006900E0F24E96E88
:103BB000070E1020EA6E0DC0EFFF900E0F26000ECC
:103BC000102201D012000FC013F010C014F00D50DD
:103BD00058D811A002D088D965DA050E636F426A01
:103BE00012000D6E9F51E96E050EA025EA6E040EBF
:103BF000EF6EEFEC0FF09F51E96E050EA025EA6E17
:103C0000B40EEF6EEFEC0FF09F51E96E050EA0259C
:103C1000EA6E6F0EEF6EEFEC0FF09F51E96E050E3E
:103C2000A025EA6E0DC0EFFFEFEC0FF09D519F5DF8
:103C30000E6E9E51A0590F6E0FAE02D0020E0F26CF
:103C40000FBE06D0E10E0E5C010E0F58D8B02D98B5
:103C500012009B2B04EE00F09B51E9266F0EEF62E1
:103C600004D0A9A102D0A991396A1200A6B2FED748
:103C700016C0A9FF17C0AAFFA69EA69CA680A850A2
:103C80001200156E13C016F014C017F0EFDF1518F0
:103C90001CE0A6B2FED715C0A8FF13C0A9FF14C030
:103CA000AAFFA69EA69CA684F29E550EA76EAA0EFB
:103CB000A76EA682F28EA69413C016F014C017F059
:103CC000D5DF151802E0D8901200D88012007FCFFF
:103CD000F6FF7FCFF7FFF86AA68EA69C0800F55086
:103CE0001200F00ED36EC00E9B6E100E386F020ED7
:103CF000396F3A6B110EC26EC16ABE0EC06E800E75
:103D0000806E200E926E816AF30E936E616A826AF3
:103D1000FC0E946E200EAC6E900EAB6E100EB86E54
:103D20003B0EAF6E0A6A0B6A2B0EC26EC2B2FED792
:103D3000030EC4140B6EC3CF0AF0220E0A5C010EF0
:103D40000B580BE2899E640E136ED5EC11F0898E30
:103D5000640E136ED5EC11F0E5D70FEE37F0ED6A77
:103D6000EA50FDE1E950FBE1EF6AF26AF16AF06ABC
:103D70009D6AA06A9F6AA26AD59ED66A340ECD6EED
:103D80009E909D80BA6A300EB16EA68EA69CF66A91
:103D9000F76AF86A0EEE00F0400E0E6E0900F5525A
:103DA000F5CFEEFF0E2EFAD70E6A12800EEE00F05F
:103DB0000E50E926EFCF0FF0D7D9106E0F501062DA
:103DC00012900E2A070E0E64F1D712B01CD00E6AA4
:103DD000080E0E600BD00E50C7D90F6E0EEE00F01D
:103DE0000E50E9260FC0EFFF0E2AF2D787D90BE25B
:103DF000899E960E136ED5EC11F0898E960E136E79
:103E0000D5EC11F0F3D70D019283130EC26E0F01A2
:103E1000C2B2FDD7030EC4140D6EC3CF0CF0010E59
:103E20000C5C030E0D5802E3D8801200D8901200EB
:103E300007EE00F00A6A0B6A0AC016F00BC017F012
:103E400015DFEE6E0A2A000E0B22980E0A5C010E98
:103E50000B58F2E392C860F093C861F094C862F026
:103E60003F0E070104150101616F05C760F1A68EC1
:103E7000A69CF66AF76A200EF86E0EEE40F0080E69
:103E8000126E0900F5CFEEFF122EFBD745CE48FE8D
:103E9000130EC26E0001C2B2FED7030EC414116E1F
:103EA000C3CF10F0869786958693200E105C010E86
:103EB000115802E2868317D0220E105C010E1158B1
:103EC00007E3800E105C010E115802E286850BD0CC
:103ED000820E105C010E115806E3800E105C020E7B
:103EE0001158D8A08687120027EE12F0156A020E2C
:103EF000156027D0010E146E02EE12F01550E9265F
:103F0000EF6A02EE00F0E926EF6ADFAC07D002EEBE
:103F100000F01550E9261450EF1209D0DCAE06D09F
:103F200002EE12F01550E9261450EF12DD50D89031
:103F30001436080ED926000EDA221466E6D7152AA2
:103F4000D6D7200E926E030E936EC00E946E156A35
:103F500002EE00F01550E926EFAE9290EFBE92808F
:103F600002EE00F0E926EFAA9292EFBA928202EEF8
:103F700000F0E926EFA69294EFB6928402EE00F0EC
:103F8000E926EFA29296EFB2928602EE00F0E926C1
:103F9000EFA49394EFB4938402EE00F0E926EFA02F
:103FA0009396EFB0938602EE00F0E926EFAC949082
:103FB000EFBC948002EE00F0E926EFA89492EFB8EF
:103FC0009482010E156E02EE00F0E926EFAE939892
:103FD000EFBE938802EE00F0E926EFAA939AEFBABB
:103FE000938A02EE00F0E926EFA6939CEFB6938C3D
:103FF00002EE00F0E926EFA2939EEFB2938E02EE5E
:1040000000F0E926EFAC9494EFBC948402EE00F04B
:10401000E926EFA89496EFB8948602EE00F0E92620
:10402000EFA49498EFB4948802EE00F0E926EFA094
:10403000949AEFB0948A120009A133D027EE11F0C0
:104040000B6A020E0B602DD0010E0D6E0C6ADFBCE8
:1040500002D00D500C12D8900D36080ED926000E45
:10406000DA220D66F4D7900E0B24E96E080EEA6A88
:10407000EA22EFCF0AF002EE08F00B50E9260C50CE
:104080000A14EF6E02EE00F00B50E926EF1C0A6EE8
:1040900002EE0EF00B50E9260C500A14EF6E0B2ABC
:1040A000D0D71200996B126A100E12600CD0080E55
:1040B0001202F350100FD96E070EDA6ADA22DF50BF
:1040C0009927122AF1D7040E01016003F350000171
:1040D00099273F0E991799C006F712000A6A99515D
:1040E0000A600BD0A192B368B26AB180A1A2FED7D8
:1040F000B1908BBF02D00A2AF2D71200020E136EC3
:10410000A68EA69CA684A68EF66AF76AF86AA6888A
:10411000550EA76EAA0EA76EA682A6980A000EEEEE
:1041200000F0400E146EEECFF5FF0F00142EFBD7FB
:10413000550EA76EAA0EA76EA682A694F66A0EEE7C
:1041400000F01580400E146E0900F550EE1802E0E4
:10415000159002D0142EF8D715A002D0D8801200E6
:10416000132ED0D7D8901200136E7C0FF66E410E2E
:10417000F76AF722F86A0800F550120000EF02F023
:0441800000EF08F054
:0200000400F00A
:1000000014571600270F00E0009F000000000000BA
:100010000020430000000000012043000000000019
:100020000220430000000000032043000000000005
:1000300004204300000000000520430000000000F1
:1000400006204300000000000720430000000000DD
:1000500008204300000000000920430000000000C9
:100060000A204300000000000B20430000000000B5
:100070000C204300000000000D20430000000000A1
:100080000E204300000000000F204300000000008D
:100090000000000000000000000000000000000060
:1000A0000000000000000000000000000000000050
:1000B0000000000000000000000000000000000040
:1000C0000000000000000000000000000000000030
:1000D0000000000000000000000000000000000020
:1000E0000000000000000000000000000000000010
:1000F0000000000000000000000000000000000000
:1001000000000000000000000000000000000000EF
:1001100000000000000000000000000000000000DF
:1001200000000000000000000000000000000000CF
:1001300000000000000000000000000000000000BF
:1001400000000000000000000000000000000000AF
:10015000000000000000000000000000000000009F
:10016000000000000000000000000000000000008F
:10017000000000000000000000000000000000007F
:10018000000000000000000000000000000000006F
:08019000000000000000000067
:020000040000FA
:0400000000EF02F01B
:020000040030CA
:0E000000FF280008FF8181FF0FC00FE00F40B6
:00000001FF
